:100000002DC047C046C045C044C043C042C041C0E7
:1000100040C03FC03EC03DC0AAC33BC03AC039C08B
:100020008BC037C036C034C3BDC1C0C1CAC1DBC17B
:10003000F8C116C228C227C2F9C103C224C223C212
:1000400022C221C220C209C20BC20AC21CC21BC2E8
:100050001AC219C218C217C216C207C211241FBE83
:10006000CFEFD2E0DEBFCDBF11E0A0E0B1E0E8EA23
:10007000F8E002C005900D92A430B107D9F721E055
:10008000A4E0B1E001C01D92A433B207E1F76DD244
:1000900009C4B6CFE4E6F0E080818E7F8083EAE792
:1000A000F0E08FED8083ACE7B0E08C918F7D8C9396
:1000B0008081886880830895282F803188F490910A
:1000C0007C00907F982B90937C00883030F481E006
:1000D00001C0880F2A95EAF701C080E080937E0076
:1000E000613021F480917C00806405C0623029F485
:1000F00080917C008F7B80937C00089590917A00A2
:10010000292F207496FD15C080930C01662311F0F1
:10011000982F01C090E09093040190917C009F7013
:10012000906890931F0190917A00906490937A0068
:1001300001C021E0822F08951F920F920FB60F92F7
:1001400011242F934F935F938F939F93AF93BF93FC
:10015000EF93FF93E0917C00EF7020910401222344
:10016000D1F080910C012817B1F0E930A0F4AE2F46
:10017000B0E0AA0FBB1FA35FBE4F4D915C911197DA
:100180008091780090917900840F951F96958795BE
:1001900011969C938E9380910C01882359F0809145
:1001A0000C01815080930C0180917A0080648093CF
:1001B0007A0011C021110DC0E93058F4F0E08091AF
:1001C000780090917900EE0FFF1FE35FFE4F91835F
:1001D000808310921F01FF91EF91BF91AF919F918A
:1001E0008F915F914F912F910F900FBE0F901F90A5
:1001F00018958AB1806F8AB987B18F6087B98BB142
:10020000806F8BB988B18F6088B90895CF93DF93E1
:100210008BB1806F8BB988B18F6088B9C8E8D0E0A6
:100220008EEF8883AAE8B0E08C938AEF90E09093F9
:100230008500809384003BB124E02D0D81E090E0A7
:10024000AC0101C0440F2A95EAF7242F20952323FF
:100250002BB928B10D2C01C0880F0A94EAF78095BC
:10026000822388B9ED2DF0E0EB5DFE4F8BEF90819E
:10027000282F291B2883ED2DF0E0EF5DFE4F9081A4
:10028000891B8C93DF91CF9108959BB1906F9BB99F
:10029000E0E8F0E090819F70908397B1907F97B9EC
:1002A00095B7906195BF47B121E030E0B90102C038
:1002B000660F771F8A95E2F7CB01462B47B998B1B5
:1002C000907F98B92A9A98B1982B98B92A9878E093
:1002D0007A95F1F797B18095982397B998B18923CA
:1002E00088B985B78F7E85BF0895843038F466233A
:1002F00029F0E82FF0E0E050FF4F6083089583700D
:1003000080930501089580910501E82FF0E0E05009
:10031000FF4F9081911101C091E02E2DE11003C09B
:1003200061E08FE012C0213019F460E080E018C075
:10033000223061F490911F01992319F0EE24E39487
:100340000895A3DF6FEF80910501B6CE4E2D50E0EA
:10035000892F90E002964817590719F461E083E06D
:10036000CDCE8417950794F42150E22E80911F0181
:1003700081110CC06FEF8FE09FDE3BDF8EEF80932B
:10038000800084B1866084B91092200108958F2D79
:100390004F2D50E04A31510508F075C0FA01EC5E6E
:1003A000FF4F0994F12C10922A0108958091330196
:1003B000882309F46CC0F090300183E0809333010E
:1003C00050C0E0912F01E43020F4F0E0EB5DFE4FEF
:1003D00006C0E83008F044C0F0E0E35EFE4F8091D4
:1003E000300180833DC080913301882309F44FC0E0
:1003F00080911D0190911E01892B09F444C06091E8
:100400001D0170911E0180913001681B710987FDEB
:10041000739570930701609306018EE390E024D2F8
:100420001FC0809133018230D8F41DC0809120011B
:10043000811117C010922001E12C88E080932001E7
:1004400010C08091200181110CC010922001E12C7C
:1004500080912F0154DF81E0F1CF84E08093090186
:10046000F12C10922A0180E00895809133018823B5
:1004700071F080912F01843098F7609130016623EC
:1004800079F333DFEDCFF12C10922A0181E008954A
:100490008093BB00ECEBF0E08081806880838081FA
:1004A0008F7B808380E008958F2D8830B9F089306C
:1004B000C1F0843051F580912F01803428F490E010
:1004C000C8D1E6DF81E006C08091BC008F7B8093BD
:1004D000BC008FEFF12C10922A0108958091080141
:1004E0000EC0E0912F01E370F0E0EE0FFF1FE35F1D
:1004F000FE4F808191819695879596958795C8DF67
:10050000F12C10922A0181E008958091BC008F7B2C
:100510008093BC008FEF089580911D0190911E0182
:1005200090910601891B982F959595959595891B16
:1005300008958E2DE11003C062E088E0BDCD8330C8
:1005400019F461E084E0DACD843070F08150E82E57
:1005500080911F01811108C061E08FE0ADDD109234
:100560002001DADF80930801089580E8809361001C
:100570001092610082B3806F82BB1DB881E084B9A4
:1005800017B81AB8CFEFCEB9DEEFD5B9C8B9CBB925
:1005900030DE22E02093B8008CEF8093B90086EE25
:1005A0008093BA001092BD0085E48093BC008091D6
:1005B00064008A7F809364009BEF95BD8DE387BDC7
:1005C00016BC20936E00809164008C7F8093640041
:1005D000C0938900C0938800C0938A001092850060
:1005E00010928400D093800089E180938100109262
:1005F000820080918000809329019093860084B1CD
:10060000866084B910926F0045DD629923C042DD97
:100610002FEF80E792E0215080409040E1F700C04A
:100620000000629917C0789488E08093200181DFF0
:1006300080911F018111FCCF60911D0170911E01FD
:1006400070930701609306018EE390E00DD1109244
:1006500020010DC08EE390E003D1813322E09207A8
:1006600014F081E191E0909307018093060183B734
:10067000897F90910901892B83BF10920901789499
:1006800083B7816083BF889583B78E7F83BFEFCFA9
:100690001F920F920FB60F9211242F933F934F93F7
:1006A0005F936F937F938F939F93AF93BF93EF93DA
:1006B000FF938091B900887F803AF1F160F4883629
:1006C00009F43FC028F4882391F18036D1F134C079
:1006D000803839F031C0883B41F170F5883A29F112
:1006E0002BC08091BB00F1100FC0982F92959F7086
:1006F000F92E982F9F7090932F0110923301109232
:100700002A0187FF1EC00AC0E0913301EF5FE3704A
:10071000E0933301F0E0E15DFE4F808338DE882313
:1007200081F08091BC008F7B0AC0BEDE0AC0809140
:10073000BC0080698093BC008091BC008064809381
:10074000BC008091BC0080688093BC00FF91EF9159
:10075000BF91AF919F918F917F916F915F914F91D9
:100760003F912F910F900FBE0F901F9018951F92E1
:100770000F920FB60F9211242F933F934F935F93D5
:100780006F937F938F939F93AF93BF93EF93FF9359
:1007900080910B018F5F883C18F480930B010CC093
:1007A00010920B0180910A018F5F843618F48093B8
:1007B0000A0102C010920A0187B58D3311F08DE352
:1007C00001C08EE387BD80912001882371F0809164
:1007D0002001813021F0883019F4ABDE01C093DDB7
:1007E0008E2D8F3F11F08F5FE82E80912001813098
:1007F00041F081E08D0D833010F4D82E01C0D12C52
:1008000005DDFF20A1F080912A018F5F80932A01EE
:10081000823368F0F12C10922A018091BC008F7B0A
:100820008093BC008091BC0080648093BC0086B53E
:10083000FF91EF91BF91AF919F918F917F916F91B8
:100840005F914F913F912F910F900FBE0F901F908E
:100850001895F999FECF81BDF89A992780B508952A
:10086000A8E1B0E042E005C010D0272F0FC0DC01A6
:10087000862FE82FF999FECF05C0E1BDF89AE395E0
:1008800000B40D924150C8F70895262FF999FECF74
:100890001FBA81BD20BD0FB6F894FA9AF99A0FBE1F
:0808A00001960895F894FFCFC2
:0408A8000101010148
:00000001FF
